
D:\STM32\Program\1.11_Odchudzanie\um0427\FWLib\project\RIDE\STM3210E-EVAL\stm32f10x_flash.o:     file format elf32-littlearm
D:\STM32\Program\1.11_Odchudzanie\um0427\FWLib\project\RIDE\STM3210E-EVAL\stm32f10x_flash.o

Disassembly of section .text.FLASH_SetLatency:

00000000 <FLASH_SetLatency>:
FLASH_SetLatency():
D:\STM32\Program\1.11_Odchudzanie\um0427\FWLib\library\src/stm32f10x_flash.c:92
   0:	4a04      	ldr	r2, [pc, #16]	(14 <FLASH_SetLatency+0x14>)
   2:	6813      	ldr	r3, [r2, #0]
   4:	f003 0338 	and.w	r3, r3, #56	; 0x38
   8:	6013      	str	r3, [r2, #0]
D:\STM32\Program\1.11_Odchudzanie\um0427\FWLib\library\src/stm32f10x_flash.c:93
   a:	6813      	ldr	r3, [r2, #0]
   c:	4318      	orrs	r0, r3
   e:	6010      	str	r0, [r2, #0]
D:\STM32\Program\1.11_Odchudzanie\um0427\FWLib\library\src/stm32f10x_flash.c:94
  10:	4770      	bx	lr
  12:	46c0      	nop			(mov r8, r8)
  14:	40022000 	.word	0x40022000
Disassembly of section .text.FLASH_HalfCycleAccessCmd:

00000000 <FLASH_HalfCycleAccessCmd>:
FLASH_HalfCycleAccessCmd():
D:\STM32\Program\1.11_Odchudzanie\um0427\FWLib\library\src/stm32f10x_flash.c:112
   0:	4a04      	ldr	r2, [pc, #16]	(14 <FLASH_HalfCycleAccessCmd+0x14>)
   2:	6813      	ldr	r3, [r2, #0]
   4:	f023 0308 	bic.w	r3, r3, #8	; 0x8
   8:	6013      	str	r3, [r2, #0]
D:\STM32\Program\1.11_Odchudzanie\um0427\FWLib\library\src/stm32f10x_flash.c:113
   a:	6813      	ldr	r3, [r2, #0]
   c:	4318      	orrs	r0, r3
   e:	6010      	str	r0, [r2, #0]
D:\STM32\Program\1.11_Odchudzanie\um0427\FWLib\library\src/stm32f10x_flash.c:114
  10:	4770      	bx	lr
  12:	46c0      	nop			(mov r8, r8)
  14:	40022000 	.word	0x40022000
Disassembly of section .text.FLASH_PrefetchBufferCmd:

00000000 <FLASH_PrefetchBufferCmd>:
FLASH_PrefetchBufferCmd():
D:\STM32\Program\1.11_Odchudzanie\um0427\FWLib\library\src/stm32f10x_flash.c:132
   0:	4a04      	ldr	r2, [pc, #16]	(14 <FLASH_PrefetchBufferCmd+0x14>)
   2:	6813      	ldr	r3, [r2, #0]
   4:	f023 0310 	bic.w	r3, r3, #16	; 0x10
   8:	6013      	str	r3, [r2, #0]
D:\STM32\Program\1.11_Odchudzanie\um0427\FWLib\library\src/stm32f10x_flash.c:133
   a:	6813      	ldr	r3, [r2, #0]
   c:	4318      	orrs	r0, r3
   e:	6010      	str	r0, [r2, #0]
D:\STM32\Program\1.11_Odchudzanie\um0427\FWLib\library\src/stm32f10x_flash.c:134
  10:	4770      	bx	lr
  12:	46c0      	nop			(mov r8, r8)
  14:	40022000 	.word	0x40022000
Disassembly of section .text.FLASH_Unlock:

00000000 <FLASH_Unlock>:
FLASH_Unlock():
D:\STM32\Program\1.11_Odchudzanie\um0427\FWLib\library\src/stm32f10x_flash.c:147
   0:	4b03      	ldr	r3, [pc, #12]	(10 <FLASH_Unlock+0x10>)
   2:	4a04      	ldr	r2, [pc, #16]	(14 <FLASH_Unlock+0x14>)
   4:	605a      	str	r2, [r3, #4]
D:\STM32\Program\1.11_Odchudzanie\um0427\FWLib\library\src/stm32f10x_flash.c:148
   6:	f102 3288 	add.w	r2, r2, #2290649224	; 0x88888888
   a:	605a      	str	r2, [r3, #4]
D:\STM32\Program\1.11_Odchudzanie\um0427\FWLib\library\src/stm32f10x_flash.c:149
   c:	4770      	bx	lr
   e:	46c0      	nop			(mov r8, r8)
  10:	40022000 	.word	0x40022000
  14:	45670123 	.word	0x45670123
Disassembly of section .text.FLASH_Lock:

00000000 <FLASH_Lock>:
FLASH_Lock():
D:\STM32\Program\1.11_Odchudzanie\um0427\FWLib\library\src/stm32f10x_flash.c:161
   0:	4a02      	ldr	r2, [pc, #8]	(c <FLASH_Lock+0xc>)
   2:	6913      	ldr	r3, [r2, #16]
   4:	f043 0380 	orr.w	r3, r3, #128	; 0x80
   8:	6113      	str	r3, [r2, #16]
D:\STM32\Program\1.11_Odchudzanie\um0427\FWLib\library\src/stm32f10x_flash.c:162
   a:	4770      	bx	lr
   c:	40022000 	.word	0x40022000
Disassembly of section .text.FLASH_GetUserOptionByte:

00000000 <FLASH_GetUserOptionByte>:
FLASH_GetUserOptionByte():
D:\STM32\Program\1.11_Odchudzanie\um0427\FWLib\library\src/stm32f10x_flash.c:665
   0:	4b01      	ldr	r3, [pc, #4]	(8 <FLASH_GetUserOptionByte+0x8>)
   2:	69d8      	ldr	r0, [r3, #28]
D:\STM32\Program\1.11_Odchudzanie\um0427\FWLib\library\src/stm32f10x_flash.c:666
   4:	0880      	lsrs	r0, r0, #2
   6:	4770      	bx	lr
   8:	40022000 	.word	0x40022000
Disassembly of section .text.FLASH_GetWriteProtectionOptionByte:

00000000 <FLASH_GetWriteProtectionOptionByte>:
FLASH_GetWriteProtectionOptionByte():
D:\STM32\Program\1.11_Odchudzanie\um0427\FWLib\library\src/stm32f10x_flash.c:678
   0:	4b01      	ldr	r3, [pc, #4]	(8 <FLASH_GetWriteProtectionOptionByte+0x8>)
   2:	6a18      	ldr	r0, [r3, #32]
D:\STM32\Program\1.11_Odchudzanie\um0427\FWLib\library\src/stm32f10x_flash.c:679
   4:	4770      	bx	lr
   6:	46c0      	nop			(mov r8, r8)
   8:	40022000 	.word	0x40022000
Disassembly of section .text.FLASH_GetReadOutProtectionStatus:

00000000 <FLASH_GetReadOutProtectionStatus>:
FLASH_GetReadOutProtectionStatus():
D:\STM32\Program\1.11_Odchudzanie\um0427\FWLib\library\src/stm32f10x_flash.c:693
   0:	4b02      	ldr	r3, [pc, #8]	(c <FLASH_GetReadOutProtectionStatus+0xc>)
   2:	69d8      	ldr	r0, [r3, #28]
D:\STM32\Program\1.11_Odchudzanie\um0427\FWLib\library\src/stm32f10x_flash.c:702
   4:	f3c0 0040 	ubfx	r0, r0, #1, #1
   8:	4770      	bx	lr
   a:	46c0      	nop			(mov r8, r8)
   c:	40022000 	.word	0x40022000
Disassembly of section .text.FLASH_GetPrefetchBufferStatus:

00000000 <FLASH_GetPrefetchBufferStatus>:
FLASH_GetPrefetchBufferStatus():
D:\STM32\Program\1.11_Odchudzanie\um0427\FWLib\library\src/stm32f10x_flash.c:715
   0:	4b02      	ldr	r3, [pc, #8]	(c <FLASH_GetPrefetchBufferStatus+0xc>)
   2:	6818      	ldr	r0, [r3, #0]
D:\STM32\Program\1.11_Odchudzanie\um0427\FWLib\library\src/stm32f10x_flash.c:725
   4:	f3c0 1040 	ubfx	r0, r0, #5, #1
   8:	4770      	bx	lr
   a:	46c0      	nop			(mov r8, r8)
   c:	40022000 	.word	0x40022000
Disassembly of section .text.FLASH_ITConfig:

00000000 <FLASH_ITConfig>:
FLASH_ITConfig():
D:\STM32\Program\1.11_Odchudzanie\um0427\FWLib\library\src/stm32f10x_flash.c:744
   0:	b121      	cbz	r1, c <FLASH_ITConfig+0xc>
D:\STM32\Program\1.11_Odchudzanie\um0427\FWLib\library\src/stm32f10x_flash.c:747
   2:	4a05      	ldr	r2, [pc, #20]	(18 <FLASH_ITConfig+0x18>)
   4:	6913      	ldr	r3, [r2, #16]
   6:	ea40 0303 	orr.w	r3, r0, r3
   a:	e003      	b.n	14 <FLASH_ITConfig+0x14>
D:\STM32\Program\1.11_Odchudzanie\um0427\FWLib\library\src/stm32f10x_flash.c:752
   c:	4a02      	ldr	r2, [pc, #8]	(18 <FLASH_ITConfig+0x18>)
   e:	6913      	ldr	r3, [r2, #16]
  10:	ea23 0300 	bic.w	r3, r3, r0
  14:	6113      	str	r3, [r2, #16]
D:\STM32\Program\1.11_Odchudzanie\um0427\FWLib\library\src/stm32f10x_flash.c:754
  16:	4770      	bx	lr
  18:	40022000 	.word	0x40022000
Disassembly of section .text.FLASH_GetFlagStatus:

00000000 <FLASH_GetFlagStatus>:
FLASH_GetFlagStatus():
D:\STM32\Program\1.11_Odchudzanie\um0427\FWLib\library\src/stm32f10x_flash.c:776
   0:	2801      	cmp	r0, #1
   2:	d104      	bne.n	e <FLASH_GetFlagStatus+0xe>
D:\STM32\Program\1.11_Odchudzanie\um0427\FWLib\library\src/stm32f10x_flash.c:778
   4:	4b05      	ldr	r3, [pc, #20]	(1c <FLASH_GetFlagStatus+0x1c>)
   6:	69db      	ldr	r3, [r3, #28]
   8:	f003 0001 	and.w	r0, r3, #1	; 0x1
   c:	e005      	b.n	1a <FLASH_GetFlagStatus+0x1a>
D:\STM32\Program\1.11_Odchudzanie\um0427\FWLib\library\src/stm32f10x_flash.c:789
   e:	4b03      	ldr	r3, [pc, #12]	(1c <FLASH_GetFlagStatus+0x1c>)
  10:	68db      	ldr	r3, [r3, #12]
  12:	4218      	tst	r0, r3
  14:	bf0c      	ite	eq
  16:	2000      	moveq	r0, #0
  18:	2001      	movne	r0, #1
D:\STM32\Program\1.11_Odchudzanie\um0427\FWLib\library\src/stm32f10x_flash.c:800
  1a:	4770      	bx	lr
  1c:	40022000 	.word	0x40022000
Disassembly of section .text.FLASH_ClearFlag:

00000000 <FLASH_ClearFlag>:
FLASH_ClearFlag():
D:\STM32\Program\1.11_Odchudzanie\um0427\FWLib\library\src/stm32f10x_flash.c:820
   0:	4b01      	ldr	r3, [pc, #4]	(8 <FLASH_ClearFlag+0x8>)
   2:	60d8      	str	r0, [r3, #12]
D:\STM32\Program\1.11_Odchudzanie\um0427\FWLib\library\src/stm32f10x_flash.c:821
   4:	4770      	bx	lr
   6:	46c0      	nop			(mov r8, r8)
   8:	40022000 	.word	0x40022000
Disassembly of section .text.FLASH_GetStatus:

00000000 <FLASH_GetStatus>:
FLASH_GetStatus():
D:\STM32\Program\1.11_Odchudzanie\um0427\FWLib\library\src/stm32f10x_flash.c:835
   0:	4a09      	ldr	r2, [pc, #36]	(28 <FLASH_GetStatus+0x28>)
   2:	68d3      	ldr	r3, [r2, #12]
   4:	f013 0f01 	tst.w	r3, #1	; 0x1
   8:	d001      	beq.n	e <FLASH_GetStatus+0xe>
   a:	2001      	movs	r0, #1
   c:	e00b      	b.n	26 <FLASH_GetStatus+0x26>
D:\STM32\Program\1.11_Odchudzanie\um0427\FWLib\library\src/stm32f10x_flash.c:841
   e:	68d3      	ldr	r3, [r2, #12]
  10:	f013 0f04 	tst.w	r3, #4	; 0x4
  14:	d001      	beq.n	1a <FLASH_GetStatus+0x1a>
  16:	2002      	movs	r0, #2
  18:	e005      	b.n	26 <FLASH_GetStatus+0x26>
D:\STM32\Program\1.11_Odchudzanie\um0427\FWLib\library\src/stm32f10x_flash.c:847
  1a:	68d3      	ldr	r3, [r2, #12]
  1c:	f013 0f10 	tst.w	r3, #16	; 0x10
  20:	bf0c      	ite	eq
  22:	2004      	moveq	r0, #4
  24:	2003      	movne	r0, #3
D:\STM32\Program\1.11_Odchudzanie\um0427\FWLib\library\src/stm32f10x_flash.c:859
  26:	4770      	bx	lr
  28:	40022000 	.word	0x40022000
Disassembly of section .text.FLASH_WaitForLastOperation:

00000000 <FLASH_WaitForLastOperation>:
FLASH_WaitForLastOperation():
D:\STM32\Program\1.11_Odchudzanie\um0427\FWLib\library\src/stm32f10x_flash.c:871
   0:	b513      	push	{r0, r1, r4, lr}
   2:	4604      	mov	r4, r0
D:\STM32\Program\1.11_Odchudzanie\um0427\FWLib\library\src/stm32f10x_flash.c:875
   4:	f7ff fffe 	bl	0 <FLASH_WaitForLastOperation>
D:\STM32\Program\1.11_Odchudzanie\um0427\FWLib\library\src/stm32f10x_flash.c:878
   8:	e00c      	b.n	24 <FLASH_WaitForLastOperation+0x24>
delay():
D:\STM32\Program\1.11_Odchudzanie\um0427\FWLib\library\src/stm32f10x_flash.c:903
   a:	2300      	movs	r3, #0
   c:	9301      	str	r3, [sp, #4]
D:\STM32\Program\1.11_Odchudzanie\um0427\FWLib\library\src/stm32f10x_flash.c:905
   e:	33ff      	adds	r3, #255
  10:	e001      	b.n	16 <FLASH_WaitForLastOperation+0x16>
  12:	9b01      	ldr	r3, [sp, #4]
  14:	3b01      	subs	r3, #1
  16:	9301      	str	r3, [sp, #4]
  18:	9b01      	ldr	r3, [sp, #4]
  1a:	2b00      	cmp	r3, #0
  1c:	d1f9      	bne.n	12 <FLASH_WaitForLastOperation+0x12>
FLASH_WaitForLastOperation():
D:\STM32\Program\1.11_Odchudzanie\um0427\FWLib\library\src/stm32f10x_flash.c:881
  1e:	f7ff fffe 	bl	0 <FLASH_WaitForLastOperation>
D:\STM32\Program\1.11_Odchudzanie\um0427\FWLib\library\src/stm32f10x_flash.c:882
  22:	3c01      	subs	r4, #1
D:\STM32\Program\1.11_Odchudzanie\um0427\FWLib\library\src/stm32f10x_flash.c:878
  24:	2801      	cmp	r0, #1
  26:	d102      	bne.n	2e <FLASH_WaitForLastOperation+0x2e>
  28:	2c00      	cmp	r4, #0
  2a:	d1ee      	bne.n	a <FLASH_WaitForLastOperation+0xa>
  2c:	e000      	b.n	30 <FLASH_WaitForLastOperation+0x30>
D:\STM32\Program\1.11_Odchudzanie\um0427\FWLib\library\src/stm32f10x_flash.c:885
  2e:	b904      	cbnz	r4, 32 <FLASH_WaitForLastOperation+0x32>
  30:	2005      	movs	r0, #5
D:\STM32\Program\1.11_Odchudzanie\um0427\FWLib\library\src/stm32f10x_flash.c:892
  32:	bd1c      	pop	{r2, r3, r4, pc}
Disassembly of section .text.FLASH_UserOptionByteConfig:

00000000 <FLASH_UserOptionByteConfig>:
FLASH_UserOptionByteConfig():
D:\STM32\Program\1.11_Odchudzanie\um0427\FWLib\library\src/stm32f10x_flash.c:619
   0:	e92d 41f0 	stmdb	sp!, {r4, r5, r6, r7, r8, lr}
D:\STM32\Program\1.11_Odchudzanie\um0427\FWLib\library\src/stm32f10x_flash.c:628
   4:	4b13      	ldr	r3, [pc, #76]	(54 <FLASH_UserOptionByteConfig+0x54>)
   6:	4c14      	ldr	r4, [pc, #80]	(58 <FLASH_UserOptionByteConfig+0x58>)
D:\STM32\Program\1.11_Odchudzanie\um0427\FWLib\library\src/stm32f10x_flash.c:619
   8:	4605      	mov	r5, r0
D:\STM32\Program\1.11_Odchudzanie\um0427\FWLib\library\src/stm32f10x_flash.c:628
   a:	60a3      	str	r3, [r4, #8]
D:\STM32\Program\1.11_Odchudzanie\um0427\FWLib\library\src/stm32f10x_flash.c:629
   c:	f103 3388 	add.w	r3, r3, #2290649224	; 0x88888888
D:\STM32\Program\1.11_Odchudzanie\um0427\FWLib\library\src/stm32f10x_flash.c:632
  10:	200f      	movs	r0, #15
D:\STM32\Program\1.11_Odchudzanie\um0427\FWLib\library\src/stm32f10x_flash.c:629
  12:	60a3      	str	r3, [r4, #8]
D:\STM32\Program\1.11_Odchudzanie\um0427\FWLib\library\src/stm32f10x_flash.c:619
  14:	460e      	mov	r6, r1
  16:	4617      	mov	r7, r2
D:\STM32\Program\1.11_Odchudzanie\um0427\FWLib\library\src/stm32f10x_flash.c:632
  18:	f7ff fffe 	bl	0 <FLASH_UserOptionByteConfig>
D:\STM32\Program\1.11_Odchudzanie\um0427\FWLib\library\src/stm32f10x_flash.c:634
  1c:	2804      	cmp	r0, #4
  1e:	d116      	bne.n	4e <FLASH_UserOptionByteConfig+0x4e>
D:\STM32\Program\1.11_Odchudzanie\um0427\FWLib\library\src/stm32f10x_flash.c:637
  20:	6923      	ldr	r3, [r4, #16]
D:\STM32\Program\1.11_Odchudzanie\um0427\FWLib\library\src/stm32f10x_flash.c:639
  22:	4a0e      	ldr	r2, [pc, #56]	(5c <FLASH_UserOptionByteConfig+0x5c>)
D:\STM32\Program\1.11_Odchudzanie\um0427\FWLib\library\src/stm32f10x_flash.c:637
  24:	f043 0310 	orr.w	r3, r3, #16	; 0x10
  28:	6123      	str	r3, [r4, #16]
D:\STM32\Program\1.11_Odchudzanie\um0427\FWLib\library\src/stm32f10x_flash.c:639
  2a:	f045 03f8 	orr.w	r3, r5, #248	; 0xf8
  2e:	ea46 0303 	orr.w	r3, r6, r3
  32:	ea47 0303 	orr.w	r3, r7, r3
D:\STM32\Program\1.11_Odchudzanie\um0427\FWLib\library\src/stm32f10x_flash.c:642
  36:	300b      	adds	r0, #11
D:\STM32\Program\1.11_Odchudzanie\um0427\FWLib\library\src/stm32f10x_flash.c:639
  38:	8053      	strh	r3, [r2, #2]
D:\STM32\Program\1.11_Odchudzanie\um0427\FWLib\library\src/stm32f10x_flash.c:642
  3a:	f7ff fffe 	bl	0 <FLASH_UserOptionByteConfig>
D:\STM32\Program\1.11_Odchudzanie\um0427\FWLib\library\src/stm32f10x_flash.c:644
  3e:	2801      	cmp	r0, #1
  40:	d005      	beq.n	4e <FLASH_UserOptionByteConfig+0x4e>
D:\STM32\Program\1.11_Odchudzanie\um0427\FWLib\library\src/stm32f10x_flash.c:647
  42:	6922      	ldr	r2, [r4, #16]
  44:	f641 73ef 	movw	r3, #8175	; 0x1fef
  48:	ea02 0303 	and.w	r3, r2, r3
  4c:	6123      	str	r3, [r4, #16]
D:\STM32\Program\1.11_Odchudzanie\um0427\FWLib\library\src/stm32f10x_flash.c:652
  4e:	e8bd 81f0 	ldmia.w	sp!, {r4, r5, r6, r7, r8, pc}
  52:	46c0      	nop			(mov r8, r8)
  54:	45670123 	.word	0x45670123
  58:	40022000 	.word	0x40022000
  5c:	1ffff800 	.word	0x1ffff800
Disassembly of section .text.FLASH_ReadOutProtection:

00000000 <FLASH_ReadOutProtection>:
FLASH_ReadOutProtection():
D:\STM32\Program\1.11_Odchudzanie\um0427\FWLib\library\src/stm32f10x_flash.c:538
   0:	b570      	push	{r4, r5, r6, lr}
   2:	4605      	mov	r5, r0
D:\STM32\Program\1.11_Odchudzanie\um0427\FWLib\library\src/stm32f10x_flash.c:544
   4:	f640 70ff 	movw	r0, #4095	; 0xfff
   8:	f7ff fffe 	bl	0 <FLASH_ReadOutProtection>
D:\STM32\Program\1.11_Odchudzanie\um0427\FWLib\library\src/stm32f10x_flash.c:546
   c:	2804      	cmp	r0, #4
   e:	d13c      	bne.n	8a <FLASH_ReadOutProtection+0x8a>
D:\STM32\Program\1.11_Odchudzanie\um0427\FWLib\library\src/stm32f10x_flash.c:549
  10:	4c1e      	ldr	r4, [pc, #120]	(8c <FLASH_ReadOutProtection+0x8c>)
  12:	4b1f      	ldr	r3, [pc, #124]	(90 <FLASH_ReadOutProtection+0x90>)
D:\STM32\Program\1.11_Odchudzanie\um0427\FWLib\library\src/stm32f10x_flash.c:556
  14:	f640 70ff 	movw	r0, #4095	; 0xfff
D:\STM32\Program\1.11_Odchudzanie\um0427\FWLib\library\src/stm32f10x_flash.c:549
  18:	60a3      	str	r3, [r4, #8]
D:\STM32\Program\1.11_Odchudzanie\um0427\FWLib\library\src/stm32f10x_flash.c:550
  1a:	f103 3388 	add.w	r3, r3, #2290649224	; 0x88888888
  1e:	60a3      	str	r3, [r4, #8]
D:\STM32\Program\1.11_Odchudzanie\um0427\FWLib\library\src/stm32f10x_flash.c:552
  20:	6923      	ldr	r3, [r4, #16]
  22:	f043 0320 	orr.w	r3, r3, #32	; 0x20
  26:	6123      	str	r3, [r4, #16]
D:\STM32\Program\1.11_Odchudzanie\um0427\FWLib\library\src/stm32f10x_flash.c:553
  28:	6923      	ldr	r3, [r4, #16]
  2a:	f043 0340 	orr.w	r3, r3, #64	; 0x40
  2e:	6123      	str	r3, [r4, #16]
D:\STM32\Program\1.11_Odchudzanie\um0427\FWLib\library\src/stm32f10x_flash.c:556
  30:	f7ff fffe 	bl	0 <FLASH_ReadOutProtection>
D:\STM32\Program\1.11_Odchudzanie\um0427\FWLib\library\src/stm32f10x_flash.c:558
  34:	2804      	cmp	r0, #4
  36:	d120      	bne.n	7a <FLASH_ReadOutProtection+0x7a>
D:\STM32\Program\1.11_Odchudzanie\um0427\FWLib\library\src/stm32f10x_flash.c:561
  38:	6923      	ldr	r3, [r4, #16]
  3a:	f641 72df 	movw	r2, #8159	; 0x1fdf
  3e:	ea03 0202 	and.w	r2, r3, r2
  42:	6122      	str	r2, [r4, #16]
D:\STM32\Program\1.11_Odchudzanie\um0427\FWLib\library\src/stm32f10x_flash.c:564
  44:	6923      	ldr	r3, [r4, #16]
  46:	f043 0310 	orr.w	r3, r3, #16	; 0x10
  4a:	6123      	str	r3, [r4, #16]
D:\STM32\Program\1.11_Odchudzanie\um0427\FWLib\library\src/stm32f10x_flash.c:566
  4c:	b11d      	cbz	r5, 56 <FLASH_ReadOutProtection+0x56>
D:\STM32\Program\1.11_Odchudzanie\um0427\FWLib\library\src/stm32f10x_flash.c:568
  4e:	4b11      	ldr	r3, [pc, #68]	(94 <FLASH_ReadOutProtection+0x94>)
  50:	f04f 0200 	mov.w	r2, #0	; 0x0
  54:	e002      	b.n	5c <FLASH_ReadOutProtection+0x5c>
D:\STM32\Program\1.11_Odchudzanie\um0427\FWLib\library\src/stm32f10x_flash.c:572
  56:	4b0f      	ldr	r3, [pc, #60]	(94 <FLASH_ReadOutProtection+0x94>)
  58:	f04f 02a5 	mov.w	r2, #165	; 0xa5
  5c:	801a      	strh	r2, [r3, #0]
D:\STM32\Program\1.11_Odchudzanie\um0427\FWLib\library\src/stm32f10x_flash.c:576
  5e:	f640 70ff 	movw	r0, #4095	; 0xfff
  62:	f7ff fffe 	bl	0 <FLASH_ReadOutProtection>
D:\STM32\Program\1.11_Odchudzanie\um0427\FWLib\library\src/stm32f10x_flash.c:578
  66:	2801      	cmp	r0, #1
  68:	d00f      	beq.n	8a <FLASH_ReadOutProtection+0x8a>
D:\STM32\Program\1.11_Odchudzanie\um0427\FWLib\library\src/stm32f10x_flash.c:581
  6a:	4908      	ldr	r1, [pc, #32]	(8c <FLASH_ReadOutProtection+0x8c>)
  6c:	f641 73ef 	movw	r3, #8175	; 0x1fef
  70:	690a      	ldr	r2, [r1, #16]
  72:	ea02 0303 	and.w	r3, r2, r3
  76:	610b      	str	r3, [r1, #16]
  78:	e007      	b.n	8a <FLASH_ReadOutProtection+0x8a>
D:\STM32\Program\1.11_Odchudzanie\um0427\FWLib\library\src/stm32f10x_flash.c:586
  7a:	2801      	cmp	r0, #1
  7c:	d005      	beq.n	8a <FLASH_ReadOutProtection+0x8a>
D:\STM32\Program\1.11_Odchudzanie\um0427\FWLib\library\src/stm32f10x_flash.c:589
  7e:	6922      	ldr	r2, [r4, #16]
  80:	f641 73df 	movw	r3, #8159	; 0x1fdf
  84:	ea02 0303 	and.w	r3, r2, r3
  88:	6123      	str	r3, [r4, #16]
D:\STM32\Program\1.11_Odchudzanie\um0427\FWLib\library\src/stm32f10x_flash.c:595
  8a:	bd70      	pop	{r4, r5, r6, pc}
  8c:	40022000 	.word	0x40022000
  90:	45670123 	.word	0x45670123
  94:	1ffff800 	.word	0x1ffff800
Disassembly of section .text.FLASH_EnableWriteProtection:

00000000 <FLASH_EnableWriteProtection>:
FLASH_EnableWriteProtection():
D:\STM32\Program\1.11_Odchudzanie\um0427\FWLib\library\src/stm32f10x_flash.c:459
   0:	b570      	push	{r4, r5, r6, lr}
   2:	4604      	mov	r4, r0
D:\STM32\Program\1.11_Odchudzanie\um0427\FWLib\library\src/stm32f10x_flash.c:474
   4:	200f      	movs	r0, #15
   6:	f7ff fffe 	bl	0 <FLASH_EnableWriteProtection>
D:\STM32\Program\1.11_Odchudzanie\um0427\FWLib\library\src/stm32f10x_flash.c:476
   a:	2804      	cmp	r0, #4
D:\STM32\Program\1.11_Odchudzanie\um0427\FWLib\library\src/stm32f10x_flash.c:474
   c:	4605      	mov	r5, r0
D:\STM32\Program\1.11_Odchudzanie\um0427\FWLib\library\src/stm32f10x_flash.c:476
   e:	d13e      	bne.n	8e <FLASH_EnableWriteProtection+0x8e>
D:\STM32\Program\1.11_Odchudzanie\um0427\FWLib\library\src/stm32f10x_flash.c:479
  10:	4a20      	ldr	r2, [pc, #128]	(94 <FLASH_EnableWriteProtection+0x94>)
  12:	4b21      	ldr	r3, [pc, #132]	(98 <FLASH_EnableWriteProtection+0x98>)
D:\STM32\Program\1.11_Odchudzanie\um0427\FWLib\library\src/stm32f10x_flash.c:467
  14:	43e4      	mvns	r4, r4
D:\STM32\Program\1.11_Odchudzanie\um0427\FWLib\library\src/stm32f10x_flash.c:479
  16:	6093      	str	r3, [r2, #8]
D:\STM32\Program\1.11_Odchudzanie\um0427\FWLib\library\src/stm32f10x_flash.c:480
  18:	f103 3388 	add.w	r3, r3, #2290649224	; 0x88888888
  1c:	6093      	str	r3, [r2, #8]
D:\STM32\Program\1.11_Odchudzanie\um0427\FWLib\library\src/stm32f10x_flash.c:481
  1e:	6913      	ldr	r3, [r2, #16]
D:\STM32\Program\1.11_Odchudzanie\um0427\FWLib\library\src/stm32f10x_flash.c:468
  20:	b2e1      	uxtb	r1, r4
D:\STM32\Program\1.11_Odchudzanie\um0427\FWLib\library\src/stm32f10x_flash.c:481
  22:	f043 0310 	orr.w	r3, r3, #16	; 0x10
D:\STM32\Program\1.11_Odchudzanie\um0427\FWLib\library\src/stm32f10x_flash.c:483
  26:	29ff      	cmp	r1, #255
D:\STM32\Program\1.11_Odchudzanie\um0427\FWLib\library\src/stm32f10x_flash.c:481
  28:	6113      	str	r3, [r2, #16]
D:\STM32\Program\1.11_Odchudzanie\um0427\FWLib\library\src/stm32f10x_flash.c:483
  2a:	d006      	beq.n	3a <FLASH_EnableWriteProtection+0x3a>
D:\STM32\Program\1.11_Odchudzanie\um0427\FWLib\library\src/stm32f10x_flash.c:485
  2c:	4b1b      	ldr	r3, [pc, #108]	(9c <FLASH_EnableWriteProtection+0x9c>)
D:\STM32\Program\1.11_Odchudzanie\um0427\FWLib\library\src/stm32f10x_flash.c:488
  2e:	200f      	movs	r0, #15
D:\STM32\Program\1.11_Odchudzanie\um0427\FWLib\library\src/stm32f10x_flash.c:485
  30:	8119      	strh	r1, [r3, #8]
D:\STM32\Program\1.11_Odchudzanie\um0427\FWLib\library\src/stm32f10x_flash.c:488
  32:	f7ff fffe 	bl	0 <FLASH_EnableWriteProtection>
D:\STM32\Program\1.11_Odchudzanie\um0427\FWLib\library\src/stm32f10x_flash.c:490
  36:	2804      	cmp	r0, #4
  38:	d11d      	bne.n	76 <FLASH_EnableWriteProtection+0x76>
D:\STM32\Program\1.11_Odchudzanie\um0427\FWLib\library\src/stm32f10x_flash.c:469
  3a:	f3c4 2207 	ubfx	r2, r4, #8, #8
D:\STM32\Program\1.11_Odchudzanie\um0427\FWLib\library\src/stm32f10x_flash.c:490
  3e:	2aff      	cmp	r2, #255
  40:	d006      	beq.n	50 <FLASH_EnableWriteProtection+0x50>
D:\STM32\Program\1.11_Odchudzanie\um0427\FWLib\library\src/stm32f10x_flash.c:492
  42:	4b16      	ldr	r3, [pc, #88]	(9c <FLASH_EnableWriteProtection+0x9c>)
D:\STM32\Program\1.11_Odchudzanie\um0427\FWLib\library\src/stm32f10x_flash.c:495
  44:	200f      	movs	r0, #15
D:\STM32\Program\1.11_Odchudzanie\um0427\FWLib\library\src/stm32f10x_flash.c:492
  46:	815a      	strh	r2, [r3, #10]
D:\STM32\Program\1.11_Odchudzanie\um0427\FWLib\library\src/stm32f10x_flash.c:495
  48:	f7ff fffe 	bl	0 <FLASH_EnableWriteProtection>
D:\STM32\Program\1.11_Odchudzanie\um0427\FWLib\library\src/stm32f10x_flash.c:498
  4c:	2804      	cmp	r0, #4
  4e:	d112      	bne.n	76 <FLASH_EnableWriteProtection+0x76>
D:\STM32\Program\1.11_Odchudzanie\um0427\FWLib\library\src/stm32f10x_flash.c:470
  50:	f3c4 4207 	ubfx	r2, r4, #16, #8
D:\STM32\Program\1.11_Odchudzanie\um0427\FWLib\library\src/stm32f10x_flash.c:498
  54:	2aff      	cmp	r2, #255
  56:	d006      	beq.n	66 <FLASH_EnableWriteProtection+0x66>
D:\STM32\Program\1.11_Odchudzanie\um0427\FWLib\library\src/stm32f10x_flash.c:500
  58:	4b10      	ldr	r3, [pc, #64]	(9c <FLASH_EnableWriteProtection+0x9c>)
D:\STM32\Program\1.11_Odchudzanie\um0427\FWLib\library\src/stm32f10x_flash.c:503
  5a:	200f      	movs	r0, #15
D:\STM32\Program\1.11_Odchudzanie\um0427\FWLib\library\src/stm32f10x_flash.c:500
  5c:	819a      	strh	r2, [r3, #12]
D:\STM32\Program\1.11_Odchudzanie\um0427\FWLib\library\src/stm32f10x_flash.c:503
  5e:	f7ff fffe 	bl	0 <FLASH_EnableWriteProtection>
D:\STM32\Program\1.11_Odchudzanie\um0427\FWLib\library\src/stm32f10x_flash.c:506
  62:	2804      	cmp	r0, #4
  64:	d107      	bne.n	76 <FLASH_EnableWriteProtection+0x76>
D:\STM32\Program\1.11_Odchudzanie\um0427\FWLib\library\src/stm32f10x_flash.c:471
  66:	0e20      	lsrs	r0, r4, #24
D:\STM32\Program\1.11_Odchudzanie\um0427\FWLib\library\src/stm32f10x_flash.c:506
  68:	28ff      	cmp	r0, #255
  6a:	d009      	beq.n	80 <FLASH_EnableWriteProtection+0x80>
D:\STM32\Program\1.11_Odchudzanie\um0427\FWLib\library\src/stm32f10x_flash.c:508
  6c:	4b0b      	ldr	r3, [pc, #44]	(9c <FLASH_EnableWriteProtection+0x9c>)
  6e:	81d8      	strh	r0, [r3, #14]
D:\STM32\Program\1.11_Odchudzanie\um0427\FWLib\library\src/stm32f10x_flash.c:511
  70:	200f      	movs	r0, #15
  72:	f7ff fffe 	bl	0 <FLASH_EnableWriteProtection>
D:\STM32\Program\1.11_Odchudzanie\um0427\FWLib\library\src/stm32f10x_flash.c:514
  76:	2801      	cmp	r0, #1
  78:	d101      	bne.n	7e <FLASH_EnableWriteProtection+0x7e>
  7a:	4605      	mov	r5, r0
  7c:	e007      	b.n	8e <FLASH_EnableWriteProtection+0x8e>
  7e:	4605      	mov	r5, r0
D:\STM32\Program\1.11_Odchudzanie\um0427\FWLib\library\src/stm32f10x_flash.c:517
  80:	4904      	ldr	r1, [pc, #16]	(94 <FLASH_EnableWriteProtection+0x94>)
  82:	f641 73ef 	movw	r3, #8175	; 0x1fef
  86:	690a      	ldr	r2, [r1, #16]
  88:	ea02 0303 	and.w	r3, r2, r3
  8c:	610b      	str	r3, [r1, #16]
D:\STM32\Program\1.11_Odchudzanie\um0427\FWLib\library\src/stm32f10x_flash.c:522
  8e:	4628      	mov	r0, r5
  90:	bd70      	pop	{r4, r5, r6, pc}
  92:	46c0      	nop			(mov r8, r8)
  94:	40022000 	.word	0x40022000
  98:	45670123 	.word	0x45670123
  9c:	1ffff800 	.word	0x1ffff800
Disassembly of section .text.FLASH_ProgramOptionByteData:

00000000 <FLASH_ProgramOptionByteData>:
FLASH_ProgramOptionByteData():
D:\STM32\Program\1.11_Odchudzanie\um0427\FWLib\library\src/stm32f10x_flash.c:410
   0:	b570      	push	{r4, r5, r6, lr}
   2:	4606      	mov	r6, r0
D:\STM32\Program\1.11_Odchudzanie\um0427\FWLib\library\src/stm32f10x_flash.c:416
   4:	200f      	movs	r0, #15
D:\STM32\Program\1.11_Odchudzanie\um0427\FWLib\library\src/stm32f10x_flash.c:410
   6:	460d      	mov	r5, r1
D:\STM32\Program\1.11_Odchudzanie\um0427\FWLib\library\src/stm32f10x_flash.c:416
   8:	f7ff fffe 	bl	0 <FLASH_ProgramOptionByteData>
D:\STM32\Program\1.11_Odchudzanie\um0427\FWLib\library\src/stm32f10x_flash.c:418
   c:	2804      	cmp	r0, #4
   e:	d115      	bne.n	3c <FLASH_ProgramOptionByteData+0x3c>
D:\STM32\Program\1.11_Odchudzanie\um0427\FWLib\library\src/stm32f10x_flash.c:421
  10:	4c0b      	ldr	r4, [pc, #44]	(40 <FLASH_ProgramOptionByteData+0x40>)
  12:	4b0c      	ldr	r3, [pc, #48]	(44 <FLASH_ProgramOptionByteData+0x44>)
D:\STM32\Program\1.11_Odchudzanie\um0427\FWLib\library\src/stm32f10x_flash.c:429
  14:	300b      	adds	r0, #11
D:\STM32\Program\1.11_Odchudzanie\um0427\FWLib\library\src/stm32f10x_flash.c:421
  16:	60a3      	str	r3, [r4, #8]
D:\STM32\Program\1.11_Odchudzanie\um0427\FWLib\library\src/stm32f10x_flash.c:422
  18:	f103 3388 	add.w	r3, r3, #2290649224	; 0x88888888
  1c:	60a3      	str	r3, [r4, #8]
D:\STM32\Program\1.11_Odchudzanie\um0427\FWLib\library\src/stm32f10x_flash.c:425
  1e:	6923      	ldr	r3, [r4, #16]
  20:	f043 0310 	orr.w	r3, r3, #16	; 0x10
  24:	6123      	str	r3, [r4, #16]
D:\STM32\Program\1.11_Odchudzanie\um0427\FWLib\library\src/stm32f10x_flash.c:426
  26:	8035      	strh	r5, [r6, #0]
D:\STM32\Program\1.11_Odchudzanie\um0427\FWLib\library\src/stm32f10x_flash.c:429
  28:	f7ff fffe 	bl	0 <FLASH_ProgramOptionByteData>
D:\STM32\Program\1.11_Odchudzanie\um0427\FWLib\library\src/stm32f10x_flash.c:431
  2c:	2801      	cmp	r0, #1
  2e:	d005      	beq.n	3c <FLASH_ProgramOptionByteData+0x3c>
D:\STM32\Program\1.11_Odchudzanie\um0427\FWLib\library\src/stm32f10x_flash.c:434
  30:	6922      	ldr	r2, [r4, #16]
  32:	f641 73ef 	movw	r3, #8175	; 0x1fef
  36:	ea02 0303 	and.w	r3, r2, r3
  3a:	6123      	str	r3, [r4, #16]
D:\STM32\Program\1.11_Odchudzanie\um0427\FWLib\library\src/stm32f10x_flash.c:439
  3c:	bd70      	pop	{r4, r5, r6, pc}
  3e:	46c0      	nop			(mov r8, r8)
  40:	40022000 	.word	0x40022000
  44:	45670123 	.word	0x45670123
Disassembly of section .text.FLASH_ProgramHalfWord:

00000000 <FLASH_ProgramHalfWord>:
FLASH_ProgramHalfWord():
D:\STM32\Program\1.11_Odchudzanie\um0427\FWLib\library\src/stm32f10x_flash.c:370
   0:	b570      	push	{r4, r5, r6, lr}
   2:	4606      	mov	r6, r0
D:\STM32\Program\1.11_Odchudzanie\um0427\FWLib\library\src/stm32f10x_flash.c:377
   4:	200f      	movs	r0, #15
D:\STM32\Program\1.11_Odchudzanie\um0427\FWLib\library\src/stm32f10x_flash.c:370
   6:	460d      	mov	r5, r1
D:\STM32\Program\1.11_Odchudzanie\um0427\FWLib\library\src/stm32f10x_flash.c:377
   8:	f7ff fffe 	bl	0 <FLASH_ProgramHalfWord>
D:\STM32\Program\1.11_Odchudzanie\um0427\FWLib\library\src/stm32f10x_flash.c:379
   c:	2804      	cmp	r0, #4
   e:	d110      	bne.n	32 <FLASH_ProgramHalfWord+0x32>
D:\STM32\Program\1.11_Odchudzanie\um0427\FWLib\library\src/stm32f10x_flash.c:382
  10:	4c08      	ldr	r4, [pc, #32]	(34 <FLASH_ProgramHalfWord+0x34>)
D:\STM32\Program\1.11_Odchudzanie\um0427\FWLib\library\src/stm32f10x_flash.c:386
  12:	300b      	adds	r0, #11
D:\STM32\Program\1.11_Odchudzanie\um0427\FWLib\library\src/stm32f10x_flash.c:382
  14:	6923      	ldr	r3, [r4, #16]
  16:	f043 0301 	orr.w	r3, r3, #1	; 0x1
  1a:	6123      	str	r3, [r4, #16]
D:\STM32\Program\1.11_Odchudzanie\um0427\FWLib\library\src/stm32f10x_flash.c:384
  1c:	8035      	strh	r5, [r6, #0]
D:\STM32\Program\1.11_Odchudzanie\um0427\FWLib\library\src/stm32f10x_flash.c:386
  1e:	f7ff fffe 	bl	0 <FLASH_ProgramHalfWord>
D:\STM32\Program\1.11_Odchudzanie\um0427\FWLib\library\src/stm32f10x_flash.c:388
  22:	2801      	cmp	r0, #1
  24:	d005      	beq.n	32 <FLASH_ProgramHalfWord+0x32>
D:\STM32\Program\1.11_Odchudzanie\um0427\FWLib\library\src/stm32f10x_flash.c:391
  26:	6922      	ldr	r2, [r4, #16]
  28:	f641 73fe 	movw	r3, #8190	; 0x1ffe
  2c:	ea02 0303 	and.w	r3, r2, r3
  30:	6123      	str	r3, [r4, #16]
D:\STM32\Program\1.11_Odchudzanie\um0427\FWLib\library\src/stm32f10x_flash.c:396
  32:	bd70      	pop	{r4, r5, r6, pc}
  34:	40022000 	.word	0x40022000
Disassembly of section .text.FLASH_ProgramWord:

00000000 <FLASH_ProgramWord>:
FLASH_ProgramWord():
D:\STM32\Program\1.11_Odchudzanie\um0427\FWLib\library\src/stm32f10x_flash.c:311
   0:	b570      	push	{r4, r5, r6, lr}
   2:	4606      	mov	r6, r0
D:\STM32\Program\1.11_Odchudzanie\um0427\FWLib\library\src/stm32f10x_flash.c:318
   4:	200f      	movs	r0, #15
D:\STM32\Program\1.11_Odchudzanie\um0427\FWLib\library\src/stm32f10x_flash.c:311
   6:	460d      	mov	r5, r1
D:\STM32\Program\1.11_Odchudzanie\um0427\FWLib\library\src/stm32f10x_flash.c:318
   8:	f7ff fffe 	bl	0 <FLASH_ProgramWord>
D:\STM32\Program\1.11_Odchudzanie\um0427\FWLib\library\src/stm32f10x_flash.c:320
   c:	2804      	cmp	r0, #4
   e:	d118      	bne.n	42 <FLASH_ProgramWord+0x42>
D:\STM32\Program\1.11_Odchudzanie\um0427\FWLib\library\src/stm32f10x_flash.c:324
  10:	4c0c      	ldr	r4, [pc, #48]	(44 <FLASH_ProgramWord+0x44>)
D:\STM32\Program\1.11_Odchudzanie\um0427\FWLib\library\src/stm32f10x_flash.c:329
  12:	300b      	adds	r0, #11
D:\STM32\Program\1.11_Odchudzanie\um0427\FWLib\library\src/stm32f10x_flash.c:324
  14:	6923      	ldr	r3, [r4, #16]
  16:	f043 0301 	orr.w	r3, r3, #1	; 0x1
  1a:	6123      	str	r3, [r4, #16]
D:\STM32\Program\1.11_Odchudzanie\um0427\FWLib\library\src/stm32f10x_flash.c:326
  1c:	b2ab      	uxth	r3, r5
  1e:	8033      	strh	r3, [r6, #0]
D:\STM32\Program\1.11_Odchudzanie\um0427\FWLib\library\src/stm32f10x_flash.c:329
  20:	f7ff fffe 	bl	0 <FLASH_ProgramWord>
D:\STM32\Program\1.11_Odchudzanie\um0427\FWLib\library\src/stm32f10x_flash.c:331
  24:	2804      	cmp	r0, #4
  26:	d104      	bne.n	32 <FLASH_ProgramWord+0x32>
D:\STM32\Program\1.11_Odchudzanie\um0427\FWLib\library\src/stm32f10x_flash.c:335
  28:	0c2b      	lsrs	r3, r5, #16
  2a:	8073      	strh	r3, [r6, #2]
D:\STM32\Program\1.11_Odchudzanie\um0427\FWLib\library\src/stm32f10x_flash.c:338
  2c:	300b      	adds	r0, #11
  2e:	f7ff fffe 	bl	0 <FLASH_ProgramWord>
D:\STM32\Program\1.11_Odchudzanie\um0427\FWLib\library\src/stm32f10x_flash.c:348
  32:	2801      	cmp	r0, #1
  34:	d005      	beq.n	42 <FLASH_ProgramWord+0x42>
D:\STM32\Program\1.11_Odchudzanie\um0427\FWLib\library\src/stm32f10x_flash.c:351
  36:	6922      	ldr	r2, [r4, #16]
  38:	f641 73fe 	movw	r3, #8190	; 0x1ffe
  3c:	ea02 0303 	and.w	r3, r2, r3
  40:	6123      	str	r3, [r4, #16]
D:\STM32\Program\1.11_Odchudzanie\um0427\FWLib\library\src/stm32f10x_flash.c:357
  42:	bd70      	pop	{r4, r5, r6, pc}
  44:	40022000 	.word	0x40022000
Disassembly of section .text.FLASH_EraseOptionBytes:

00000000 <FLASH_EraseOptionBytes>:
FLASH_EraseOptionBytes():
D:\STM32\Program\1.11_Odchudzanie\um0427\FWLib\library\src/stm32f10x_flash.c:248
   0:	b510      	push	{r4, lr}
D:\STM32\Program\1.11_Odchudzanie\um0427\FWLib\library\src/stm32f10x_flash.c:252
   2:	f640 70ff 	movw	r0, #4095	; 0xfff
   6:	f7ff fffe 	bl	0 <FLASH_EraseOptionBytes>
D:\STM32\Program\1.11_Odchudzanie\um0427\FWLib\library\src/stm32f10x_flash.c:254
   a:	2804      	cmp	r0, #4
   c:	d12c      	bne.n	68 <FLASH_EraseOptionBytes+0x68>
D:\STM32\Program\1.11_Odchudzanie\um0427\FWLib\library\src/stm32f10x_flash.c:257
   e:	4c17      	ldr	r4, [pc, #92]	(6c <FLASH_EraseOptionBytes+0x6c>)
  10:	4b17      	ldr	r3, [pc, #92]	(70 <FLASH_EraseOptionBytes+0x70>)
D:\STM32\Program\1.11_Odchudzanie\um0427\FWLib\library\src/stm32f10x_flash.c:265
  12:	f640 70ff 	movw	r0, #4095	; 0xfff
D:\STM32\Program\1.11_Odchudzanie\um0427\FWLib\library\src/stm32f10x_flash.c:257
  16:	60a3      	str	r3, [r4, #8]
D:\STM32\Program\1.11_Odchudzanie\um0427\FWLib\library\src/stm32f10x_flash.c:258
  18:	f103 3388 	add.w	r3, r3, #2290649224	; 0x88888888
  1c:	60a3      	str	r3, [r4, #8]
D:\STM32\Program\1.11_Odchudzanie\um0427\FWLib\library\src/stm32f10x_flash.c:261
  1e:	6923      	ldr	r3, [r4, #16]
  20:	f043 0320 	orr.w	r3, r3, #32	; 0x20
  24:	6123      	str	r3, [r4, #16]
D:\STM32\Program\1.11_Odchudzanie\um0427\FWLib\library\src/stm32f10x_flash.c:262
  26:	6923      	ldr	r3, [r4, #16]
  28:	f043 0340 	orr.w	r3, r3, #64	; 0x40
  2c:	6123      	str	r3, [r4, #16]
D:\STM32\Program\1.11_Odchudzanie\um0427\FWLib\library\src/stm32f10x_flash.c:265
  2e:	f7ff fffe 	bl	0 <FLASH_EraseOptionBytes>
D:\STM32\Program\1.11_Odchudzanie\um0427\FWLib\library\src/stm32f10x_flash.c:267
  32:	2804      	cmp	r0, #4
  34:	d110      	bne.n	58 <FLASH_EraseOptionBytes+0x58>
D:\STM32\Program\1.11_Odchudzanie\um0427\FWLib\library\src/stm32f10x_flash.c:270
  36:	6922      	ldr	r2, [r4, #16]
  38:	f641 73df 	movw	r3, #8159	; 0x1fdf
  3c:	ea02 0303 	and.w	r3, r2, r3
  40:	6123      	str	r3, [r4, #16]
D:\STM32\Program\1.11_Odchudzanie\um0427\FWLib\library\src/stm32f10x_flash.c:273
  42:	6923      	ldr	r3, [r4, #16]
D:\STM32\Program\1.11_Odchudzanie\um0427\FWLib\library\src/stm32f10x_flash.c:276
  44:	f04f 02a5 	mov.w	r2, #165	; 0xa5
D:\STM32\Program\1.11_Odchudzanie\um0427\FWLib\library\src/stm32f10x_flash.c:273
  48:	f043 0310 	orr.w	r3, r3, #16	; 0x10
  4c:	6123      	str	r3, [r4, #16]
D:\STM32\Program\1.11_Odchudzanie\um0427\FWLib\library\src/stm32f10x_flash.c:276
  4e:	4b09      	ldr	r3, [pc, #36]	(74 <FLASH_EraseOptionBytes+0x74>)
D:\STM32\Program\1.11_Odchudzanie\um0427\FWLib\library\src/stm32f10x_flash.c:279
  50:	300b      	adds	r0, #11
D:\STM32\Program\1.11_Odchudzanie\um0427\FWLib\library\src/stm32f10x_flash.c:276
  52:	801a      	strh	r2, [r3, #0]
D:\STM32\Program\1.11_Odchudzanie\um0427\FWLib\library\src/stm32f10x_flash.c:279
  54:	f7ff fffe 	bl	0 <FLASH_EraseOptionBytes>
D:\STM32\Program\1.11_Odchudzanie\um0427\FWLib\library\src/stm32f10x_flash.c:289
  58:	2801      	cmp	r0, #1
  5a:	d005      	beq.n	68 <FLASH_EraseOptionBytes+0x68>
D:\STM32\Program\1.11_Odchudzanie\um0427\FWLib\library\src/stm32f10x_flash.c:292
  5c:	6922      	ldr	r2, [r4, #16]
  5e:	f641 73ef 	movw	r3, #8175	; 0x1fef
  62:	ea02 0303 	and.w	r3, r2, r3
  66:	6123      	str	r3, [r4, #16]
D:\STM32\Program\1.11_Odchudzanie\um0427\FWLib\library\src/stm32f10x_flash.c:298
  68:	bd10      	pop	{r4, pc}
  6a:	46c0      	nop			(mov r8, r8)
  6c:	40022000 	.word	0x40022000
  70:	45670123 	.word	0x45670123
  74:	1ffff800 	.word	0x1ffff800
Disassembly of section .text.FLASH_EraseAllPages:

00000000 <FLASH_EraseAllPages>:
FLASH_EraseAllPages():
D:\STM32\Program\1.11_Odchudzanie\um0427\FWLib\library\src/stm32f10x_flash.c:213
   0:	b510      	push	{r4, lr}
D:\STM32\Program\1.11_Odchudzanie\um0427\FWLib\library\src/stm32f10x_flash.c:217
   2:	f640 70ff 	movw	r0, #4095	; 0xfff
   6:	f7ff fffe 	bl	0 <FLASH_EraseAllPages>
D:\STM32\Program\1.11_Odchudzanie\um0427\FWLib\library\src/stm32f10x_flash.c:219
   a:	2804      	cmp	r0, #4
   c:	d114      	bne.n	38 <FLASH_EraseAllPages+0x38>
D:\STM32\Program\1.11_Odchudzanie\um0427\FWLib\library\src/stm32f10x_flash.c:222
   e:	4c0b      	ldr	r4, [pc, #44]	(3c <FLASH_EraseAllPages+0x3c>)
D:\STM32\Program\1.11_Odchudzanie\um0427\FWLib\library\src/stm32f10x_flash.c:226
  10:	f640 70ff 	movw	r0, #4095	; 0xfff
D:\STM32\Program\1.11_Odchudzanie\um0427\FWLib\library\src/stm32f10x_flash.c:222
  14:	6923      	ldr	r3, [r4, #16]
  16:	f043 0304 	orr.w	r3, r3, #4	; 0x4
  1a:	6123      	str	r3, [r4, #16]
D:\STM32\Program\1.11_Odchudzanie\um0427\FWLib\library\src/stm32f10x_flash.c:223
  1c:	6923      	ldr	r3, [r4, #16]
  1e:	f043 0340 	orr.w	r3, r3, #64	; 0x40
  22:	6123      	str	r3, [r4, #16]
D:\STM32\Program\1.11_Odchudzanie\um0427\FWLib\library\src/stm32f10x_flash.c:226
  24:	f7ff fffe 	bl	0 <FLASH_EraseAllPages>
D:\STM32\Program\1.11_Odchudzanie\um0427\FWLib\library\src/stm32f10x_flash.c:228
  28:	2801      	cmp	r0, #1
  2a:	d005      	beq.n	38 <FLASH_EraseAllPages+0x38>
D:\STM32\Program\1.11_Odchudzanie\um0427\FWLib\library\src/stm32f10x_flash.c:231
  2c:	6922      	ldr	r2, [r4, #16]
  2e:	f641 73fb 	movw	r3, #8187	; 0x1ffb
  32:	ea02 0303 	and.w	r3, r2, r3
  36:	6123      	str	r3, [r4, #16]
D:\STM32\Program\1.11_Odchudzanie\um0427\FWLib\library\src/stm32f10x_flash.c:236
  38:	bd10      	pop	{r4, pc}
  3a:	46c0      	nop			(mov r8, r8)
  3c:	40022000 	.word	0x40022000
Disassembly of section .text.FLASH_ErasePage:

00000000 <FLASH_ErasePage>:
FLASH_ErasePage():
D:\STM32\Program\1.11_Odchudzanie\um0427\FWLib\library\src/stm32f10x_flash.c:174
   0:	b570      	push	{r4, r5, r6, lr}
   2:	4605      	mov	r5, r0
D:\STM32\Program\1.11_Odchudzanie\um0427\FWLib\library\src/stm32f10x_flash.c:181
   4:	f640 70ff 	movw	r0, #4095	; 0xfff
   8:	f7ff fffe 	bl	0 <FLASH_ErasePage>
D:\STM32\Program\1.11_Odchudzanie\um0427\FWLib\library\src/stm32f10x_flash.c:183
   c:	2804      	cmp	r0, #4
   e:	d115      	bne.n	3c <FLASH_ErasePage+0x3c>
D:\STM32\Program\1.11_Odchudzanie\um0427\FWLib\library\src/stm32f10x_flash.c:186
  10:	4c0b      	ldr	r4, [pc, #44]	(40 <FLASH_ErasePage+0x40>)
D:\STM32\Program\1.11_Odchudzanie\um0427\FWLib\library\src/stm32f10x_flash.c:191
  12:	f640 70ff 	movw	r0, #4095	; 0xfff
D:\STM32\Program\1.11_Odchudzanie\um0427\FWLib\library\src/stm32f10x_flash.c:186
  16:	6923      	ldr	r3, [r4, #16]
  18:	f043 0302 	orr.w	r3, r3, #2	; 0x2
  1c:	6123      	str	r3, [r4, #16]
D:\STM32\Program\1.11_Odchudzanie\um0427\FWLib\library\src/stm32f10x_flash.c:187
  1e:	6165      	str	r5, [r4, #20]
D:\STM32\Program\1.11_Odchudzanie\um0427\FWLib\library\src/stm32f10x_flash.c:188
  20:	6923      	ldr	r3, [r4, #16]
  22:	f043 0340 	orr.w	r3, r3, #64	; 0x40
  26:	6123      	str	r3, [r4, #16]
D:\STM32\Program\1.11_Odchudzanie\um0427\FWLib\library\src/stm32f10x_flash.c:191
  28:	f7ff fffe 	bl	0 <FLASH_ErasePage>
D:\STM32\Program\1.11_Odchudzanie\um0427\FWLib\library\src/stm32f10x_flash.c:193
  2c:	2801      	cmp	r0, #1
  2e:	d005      	beq.n	3c <FLASH_ErasePage+0x3c>
D:\STM32\Program\1.11_Odchudzanie\um0427\FWLib\library\src/stm32f10x_flash.c:196
  30:	6922      	ldr	r2, [r4, #16]
  32:	f641 73fd 	movw	r3, #8189	; 0x1ffd
  36:	ea02 0303 	and.w	r3, r2, r3
  3a:	6123      	str	r3, [r4, #16]
D:\STM32\Program\1.11_Odchudzanie\um0427\FWLib\library\src/stm32f10x_flash.c:201
  3c:	bd70      	pop	{r4, r5, r6, pc}
  3e:	46c0      	nop			(mov r8, r8)
  40:	40022000 	.word	0x40022000
